** EXPERIMENTAL (HLL) ** Open Watcom Linker Version 1.6beta1 Limited Availability
Portions Copyright (c) 1985-2002 Sybase, Inc. All Rights Reserved.
Created on:       13/11/17 16:25:32
Warning! W1121: file U:/tmp\ldconv_bz2module_obj_1aa352885a5217a508.obj(U:\DEV\python-2.7.5\Modules\bz2module.c): '_initbz2' has already been exported
Executable Image: build/lib.os2knix-2.7/bz2.pyd
creating an OS/2 EMX dynamic link library


                        +------------+
                        |   Groups   |
                        +------------+

Group                           Address              Size
=====                           =======              ====

CGROUP                          0001:00000000        00011c40
DGROUP                          0002:00000000        00002590



                        +--------------+
                        |   Segments   |
                        +--------------+

Segment                Class          Group          Address         Size
=======                =====          =====          =======         ====

TEXT32                 CODE           CGROUP         0001:00000000   00011c40
________TEXT           CODE           CGROUP         0001:00011c40   00000000
DATA32                 DATA           DGROUP         0002:00000000   00002510
SET1__os2dll           DATA           DGROUP         0002:00002510   00000004
SET2__os2dll           DATA           DGROUP         0002:00002514   00000000
SET3__os2dll           DATA           DGROUP         0002:00002514   00000004
SET1___CTOR_LIST__     DATA           DGROUP         0002:00002518   00000004
SET2___CTOR_LIST__     DATA           DGROUP         0002:0000251c   00000000
SET3___CTOR_LIST__     DATA           DGROUP         0002:0000251c   00000004
SET1___DTOR_LIST__     DATA           DGROUP         0002:00002520   00000004
SET2___DTOR_LIST__     DATA           DGROUP         0002:00002524   00000000
SET3___DTOR_LIST__     DATA           DGROUP         0002:00002524   00000004
SET1___crtinit1__      DATA           DGROUP         0002:00002528   00000004
SET2___crtinit1__      DATA           DGROUP         0002:0000252c   00000000
SET3___crtinit1__      DATA           DGROUP         0002:0000252c   00000004
SET1___crtexit1__      DATA           DGROUP         0002:00002530   00000004
SET2___crtexit1__      DATA           DGROUP         0002:00002534   00000000
SET3___crtexit1__      DATA           DGROUP         0002:00002534   00000004
SET1___eh_frame__      DATA           DGROUP         0002:00002538   00000004
SET2___eh_frame__      DATA           DGROUP         0002:0000253c   00000008
SET3___eh_frame__      DATA           DGROUP         0002:00002544   00000004
SET1___eh_init__       DATA           DGROUP         0002:00002548   00000004
SET2___eh_init__       DATA           DGROUP         0002:0000254c   00000004
SET3___eh_init__       DATA           DGROUP         0002:00002550   00000004
SET1___eh_term__       DATA           DGROUP         0002:00002554   00000004
SET2___eh_term__       DATA           DGROUP         0002:00002558   00000004
SET3___eh_term__       DATA           DGROUP         0002:0000255c   00000004
SET1___fork_parent1__  DATA           DGROUP         0002:00002560   00000004
SET2___fork_parent1__  DATA           DGROUP         0002:00002564   00000000
SET3___fork_parent1__  DATA           DGROUP         0002:00002564   00000004
SET1___fork_child1__   DATA           DGROUP         0002:00002568   00000004
SET2___fork_child1__   DATA           DGROUP         0002:0000256c   00000000
SET3___fork_child1__   DATA           DGROUP         0002:0000256c   00000004
________DATA           DATA           DGROUP         0002:00002570   00000000
BSS32                  BSS            DGROUP         0002:00002570   00000020
c_common               BSS            DGROUP         0002:00002590   00000000
________BSS            BSS            DGROUP         0002:00002590   00000000


                        +----------------+
                        |   Memory Map   |
                        +----------------+

* = unreferenced symbol
+ = symbol only referenced locally

Address        Symbol
=======        ======

Module: U:\usr\lib\dll0hi.obj({standard input})
0001:00000000* __text
0002:00000000* __data
0002:00000000* ___data_start
0002:00002570* ___bss_start
0002:00002510+ __os2dll
0002:00002518  ___CTOR_LIST__
0002:00002520  ___DTOR_LIST__
0002:00002528* ___crtinit1__
0002:00002530* ___crtexit1__
0002:00002538  ___eh_frame__
0002:00002548  ___eh_init__
0002:00002554  ___eh_term__
0002:00002560+ ___fork_parent1__
0002:00002568+ ___fork_child1__
Module: U:/tmp\ldconv_bz2module_obj_1aa352885a5217a508.obj(U:\DEV\python-2.7.5\Modules\bz2module.c)
0001:00002d38* _Util_UnivNewlineRead
0001:000041d0  _initbz2
Module: U:\usr\local473\lib\libc_dll.lib(dllinit.obj)
0001:00004460  _DLL_InitTerm
Module: U:\usr\lib\libend.lib(src/libend/386/endlink386.asm)
0002:00002590  _end
0002:00002570  _edata
Module: U:\usr\lib\libend.lib(src/libend/386/end.asm)
0001:00011c40* _etext
0001:00011c40* __etext
0000:00000000* WEAK$ZERO
0002:00002590  __end
0002:00002570  __edata
Module: U:\extras\lib\libbz2.lib(bzlib.obj)
0001:000044c0  _BZ2_bzCompressInit
0001:00004808  _BZ2_bzCompressEnd
0001:0000488c  _BZ2_bzDecompressInit
0001:00004984  _BZ2_indexIntoF
0001:000049b8  _BZ2_bzDecompressEnd
0001:00004a48* _BZ2_bzReadGetUnused
0001:00004ae4* _BZ2_bzlibVersion
0001:00004af0* _BZ2_bzflush
0001:00004af8* _BZ2_bzerror
0001:00004b50  _BZ2_bzReadClose
0001:00004bf8  _BZ2_bzReadOpen
0001:00004d88  _BZ2_bzWriteOpen
0001:0000515c* _BZ2_bzdopen
0001:00005188* _BZ2_bzopen
0001:00005214  _BZ2_bzDecompress
0001:00006068* _BZ2_bzBuffToBuffDecompress
0001:00006158  _BZ2_bzRead
0001:00006354* _BZ2_bzread
0001:00006718  _BZ2_bzCompress
0001:0000684c* _BZ2_bzBuffToBuffCompress
0001:0000694c* _BZ2_bzWriteClose64
0001:00006b74  _BZ2_bzWriteClose
0001:00006bb4* _BZ2_bzclose
0001:00006c54  _BZ2_bzWrite
0001:00006dd8* _BZ2_bzwrite
0001:000073f4  _BZ2_bz__AssertH__fail
Module: U:\tmp\ldconv_libgcc_a_1aa352885a52183590.lib(_chkstk_ms.obj)
0001:00007520  ___chkstk_ms
Module: U:\tmp\ldconv_libgcc_so_d_a_1aa352885a53159d80.lib(emx-ctordtor.obj)
0001:00007550  ___ctordtorInit
0001:00007584  ___ctordtorTerm
Module: U:\extras\lib\libbz2.lib(crctable.obj)
0002:000018a0  _BZ2_crc32Table
Module: U:\tmp\ldconv_libgcc_a_1aa352885a52183590.lib(_alloca.obj)
0001:000075c0  __alloca
Module: U:\extras\lib\libbz2.lib(decompress.obj)
0001:0000760c  _BZ2_decompress
Module: U:\extras\lib\libbz2.lib(randtable.obj)
0002:00001ca0  _BZ2_rNums
Module: U:\extras\lib\libbz2.lib(compress.obj)
0001:00009750* _BZ2_bsInitWrite
0001:00009aec  _BZ2_compressBlock
Module: U:\tmp\ldconv_libgcc_so_d_a_1aa352885a53159d80.lib(emx-eh.obj)
0001:0000e630  ___ehInit
0001:0000e666* ___ehTerm
Module: U:\extras\lib\libbz2.lib(huffman.obj)
0001:0000e6a0  _BZ2_hbAssignCodes
0001:0000e6e8  _BZ2_hbCreateDecodeTables
0001:0000e804  _BZ2_hbMakeCodeLengths
Module: U:\extras\lib\libbz2.lib(blocksort.obj)
0001:00011a40  _BZ2_blockSort


                        +----------------------+
                        |   Imported Symbols   |
                        +----------------------+

Symbol                              Module
======                              ======

___libc_ForkRegisterModule          libc065
___init_dll                         libc065
___libc_Back_termDll                libc065
___libc_ForkDeregisterModule        libc065
__atfork_callback                   libc065
_PyObject_GetAttrString             python27
_PyExc_SystemError                  python27
_PyErr_Format                       python27
_Py_BuildValue                      python27
__Py_NoneStruct                     python27
_PyString_FromString                python27
_PyInt_FromLong                     python27
_PyObject_CallMethod                python27
_PyThread_free_lock                 python27
_PyExc_ValueError                   python27
_PyErr_SetString                    python27
_PyLong_FromLongLong                python27
_PyFile_DecUseCount                 python27
_PyMem_Free                         python27
_PyThread_acquire_lock              python27
_PyThread_release_lock              python27
_PyEval_SaveThread                  python27
_PyEval_RestoreThread               python27
_PyExc_RuntimeError                 python27
_PyErr_NoMemory                     python27
_PyExc_IOError                      python27
_PyExc_EOFError                     python27
_PyArg_ParseTupleAndKeywords        python27
_PyFile_Type                        python27
_PyObject_CallFunction              python27
_PyThread_allocate_lock             python27
_PyFile_AsFile                      python27
_PyFile_IncUseCount                 python27
_PyExc_MemoryError                  python27
_PyArg_ParseTuple                   python27
_PyString_FromStringAndSize         python27
_PyExc_OverflowError                python27
_PyBuffer_Release                   python27
__PyString_Resize                   python27
_PyList_GetSlice                    python27
_PyObject_AsCharBuffer              python27
_PyList_SetItem                     python27
_PyIter_Next                        python27
_PyErr_Occurred                     python27
_PyObject_GetIter                   python27
_PyList_New                         python27
_PyExc_TypeError                    python27
_PyInt_AsLong                       python27
_PyLong_AsLongLong                  python27
_PyList_Append                      python27
_PyString_Concat                    python27
_PyMem_Malloc                       python27
_PyType_Ready                       python27
_Py_InitModule4                     python27
_PyModule_AddObject                 python27
_PyObject_GenericGetAttr            python27
_PyObject_GenericSetAttr            python27
_PyType_GenericAlloc                python27
_PyType_GenericNew                  python27
_PyObject_Free                      python27
__CRT_init                          libc065
__CRT_term                          libc065
___libc_GLocaleCtype                libc065
___stdoutp                          libc065
___stdinp                           libc065
___stderrp                          libc065
__std_memchr                        libc065
__std_memmove                       libc065
__std_memcpy                        libc065
___ctordtorInit1                    libc065
___ctordtorTerm1                    libc065
__std_fgetc                         libc065
__std_ungetc                        libc065
__std_free                          libc065
__std_malloc                        libc065
__std_strcat                        libc065
__std_fclose                        libc065
__std_fdopen                        libc065
__std_fopen                         libc065
__std_fputc                         libc065
__std_fprintf                       libc065
__std_fread                         libc065
__std_fflush                        libc065
__std_fwrite                        libc065
__std_exit                          libc065
___register_frame_table             gcc473
___deregister_frame                 gcc473


                        +--------------------+
                        |   Libraries Used   |
                        +--------------------+

U:\extras\lib\libbz2.lib
U:\tmp\ldconv_python2_7_dll_a_1aa352885a5217ef40.lib
U:\tmp\ldconv_libgcc_a_1aa352885a52183590.lib
U:\tmp\ldconv_libgcc_so_d_a_1aa352885a53159d80.lib
U:\usr\lib\libc_alias.lib
U:\usr\local473\lib\libc_dll.lib
U:\usr\lib\libend.lib


                        +-----------------------+
                        |   Linker Statistics   |
                        +-----------------------+

Stack size:  0000 (0.)
Memory size:  000141d0 (82384.)
Link time: 00:00.06
